:030000000210E308
:03000B000200A54B
:03002B000202AE20
:03005B0002040C90
:030073000203E69F
:1000800002030406080C10182030406080040608A3
:100090000C10182030406080A0C00D0D0405060D26
:1000A0000503030302C2AFC0D0C0E020620C206889
:1000B00002419D306602415DE47385258AC262E596
:1000C00025F4700221242068022111207210758B02
:1000D00000D0E0D0D0C290C291C292D2AF32C290D2
:1000E000C291C2927401D5E0FDE53C1420E21520D6
:1000F000E10D207D02C295307D02C293020121C232
:1001000094020121207D02C293307D02C29502013A
:1001100021758B00D0E0D0D0C290C291C292D2AFF4
:1001200032758B00D0E0D0D0D2AF32419DE5256052
:100130000A207D02D290307D02D292C291419DE58B
:10014000256002D291207D02C292307D02C2904190
:100150009DE525600A207D02D292307D02D290205A
:100160007D02C290307D02C292419D207D02D293D9
:10017000307D02D295207D02D295307D02D29374DB
:1001800005D5E0FDE525600A207D02D290307D0294
:10019000D292C291419D207D02D293307D02D295B0
:1001A000D2947405D5E0FDE525600A207D02D29049
:1001B000307D02D292C291419DD294207D02D29391
:1001C000307D02D2957405D5E0FDE5256002D2911F
:1001D000207D02C292307D02C290419DD294207D4A
:1001E00002D295307D02D2937405D5E0FDE52560FD
:1001F00002D291207D02C292307D02C290419D20A8
:100200007D02D295307D02D293D2947405D5E0FD63
:10021000E525600A207D02D292307D02D290207DB9
:1002200002C290307D02C292419D207D02D2953063
:100230007D02D293207D02D293307D02D295740547
:10024000D5E0FDE525600A207D02D292307D02D204
:1002500090207D02C290307D02C292419D30723D5D
:10026000E53C20E21A20E129207D02D293307D0274
:10027000D295207D02D295307D02D29302029D203C
:10028000E1E6207D02D293307D02D295D294020223
:100290009DD294207D02D295307D02D293E525F443
:1002A000F58A758B00D262D0E0D0D0D2AF32C2AF27
:1002B000C2AD53E6EFC0D0C0E0D2D3D2AFC2CEE5DC
:1002C0002960072074461529610C78007900E580C3
:1002D000307E01F430E70278FF53DACF207E03430B
:1002E000DA20307E0343DA10C2D8C271E580307E56
:1002F00001F430E70279FFC3E89970CE30610375ED
:1003000029182074037529188859D270E52A6004C9
:10031000152A611C20740543DA01C2D820700261DD
:1003200083A859206102C2702074367982B70431E3
:10033000C3E894F0400374F0F8E8C4540F28F87947
:1003400084B703026161C313C3138721200802C36A
:1003500013200A06C3C898F8616128F8500374FF97
:10036000F88822306915E5222408F5225003752209
:10037000FFC3E522955E4003855E227882B60418AD
:10038000852224A824C3E524955E4002A85EC3E824
:1003900095604002A8608825C3E52594404002D2BC
:1003A0006420CF0CD0E0D0D0C2D343E610D2AD321F
:1003B000C2CF7801E52960053074021529C3E559DB
:1003C00094014005755C0061DA755D00756400E5B7
:1003D0005C2401F55C5003755CFFD0E0D0D0C2D343
:1003E00043E610D2AD32C0D0C0E0C2AF53917F53CC
:1003F000E67FC260759100C3E49550F594E4955191
:10040000F595759104D0E0D0D0D2AF32C2AF53E6AB
:10041000EFC2ADC0D0C0E0C0F0D2D3D2AFA8FBA92C
:10042000FCC2D8307102817353DACF207E0343DAE5
:1004300010307E0343DA20D271E580307E01F42053
:10044000E702814A88268927C1AF53DACF207E038D
:1004500043DA20307E0343DA10C2D8C2713074020E
:10046000C19B7800E580307E01F430E702C19B88B3
:0F04700059C18253DACF207E0343DA20307E0356
:10047F0043DA10C271206102A14353DACF207E0309
:10048F0043DA10307E0343DA20C2D8D27188548900
:10049F0055C3E89552F8E99553F9E4FB7E027A00CB
:1004AF00C3E8948CE994005005755800A133C3E854
:1004BF0094C8E994005008E4D2E4FB7A0AA110C36F
:1004CF00E89468E994015008E4D2E3FB7A0FA11095
:1004DF00C3E894D0E994025008E4D2E2FB7A1EA15B
:1004EF0010C3E894A0E994055008E4D2E1FB7A3CEC
:1004FF00A110C3E89498E994085008E4D2E0FB7A7D
:10050F00787E00C3E89556FCE99557FD30E708EC77
:10051F00F42401FCEDF4FD755800C3EC9AED9E50E8
:10052F000375580188568957A854A955885289537D
:10053F007802C182C3E89526F8E99527F9307C0245
:10054F00C166307B02C166307A02C15F207502A19D
:10055F0066E9FDE8FCA185E9C313F9E813F83079E2
:10056F0002C15FE9C313F9E813F8307802C15FE9FC
:10057F00C313FDE813FC206126C3EC941CED940219
:10058F004002A19CED7018C3EC94C850120528C30B
:10059F00E528940A5002C19B755900D270C19BE5A2
:1005AF0028600215287400207F0B7888E67896B4AF
:1005BF000302789EE624FAFEE43400FFC3EC9EFCAF
:1005CF00ED9FFD92087888E6B40327A20850092012
:1005DF007D20C2AFD27DA1EE307D17C2AFC27DC2EA
:1005EF0090C291C292D293D294D295206902D26BCB
:1005FF00D2AFA2085017E6B4030DECF42401FCEDC2
:10060F00F43400FD02061C78007900C1667888E694
:10061F00B40315EC33FCED33FDC3EC940AFCED94FD
:10062F0000FD50047C007D00C3EC94FFED9400406E
:10063F000678FF7900C166EC856FF0A4C5F0A2F7CC
:10064F0033F87900400302068278FF7900020682B0
:10065F00E9C313F9E813F8307C0EE9600278FFC3A1
:10066F00E81338F8E43400F9C3E894FFE994004044
:10067F000278FF8859D270206102C19B741FF45514
:10068F002F4BF52FC274E42B7002D27475291830DA
:10069F00740375290A306102C1AF20740353DAFE67
:1006AF00752A06307403752A0AD0F0D0E0D0D0C274
:1006BF00D3D2AD43E6103279010206E47903020684
:1006CF00E4790A0206E4791E0206E479640206E47C
:1006DF0079C80206E47817E4D5E0FDD8FAD9F622F6
:1006EF007A147B7802070B7A107B8C02070B7A0D3A
:1006FF007BB402070B7A0B7BC802070BAC25752561
:10070F00017902B27DE4D294D5E0FDE5256002D2F5
:10071F0091D5E0FDC291D5E0FDC294D5E0FDE52570
:10072F00600A207D02D290307D02D292E570D5E032
:10073F00FD207D02C290307D02C2927496D5E0FDFD
:10074F00D9C1EAF8D5E0FDD8FBDBB1D2948C2522D4
:10075F00C37C007D0075F00005F0EA33FAEB33FB44
:10076F0050F6EB13FBEA13FAC3E9FFE8FEE89AF839
:10077F00E99BF95004EFF9EEF8B3EC33FCED33FDE0
:10078F00D5F0DFEDF9ECF822E889F08A20D2D4F821
:10079F00A9F07B0030F70B7BFFF42401F8E9F43468
:1007AF0000F9E88520F0A4ADF0F8E98520F0A4AFBA
:1007BF00F0FEED2EF974003FFA7C04C3EA13FAE958
:1007CF0013F9E813F8DCF48BF030F70AE8F424019E
:1007DF00F8E9F43400F9E889F0C2D4F8A9F02278E6
:1007EF0082B6040302084BC3E55994014003020883
:1007FF0013852224E4F53EF53FF540F541F542F52A
:10080F004702084B7882E6FC754701E522F523780D
:10081F003879C7AA3AAB3BC3EB13FBEA13FAEC14D4
:10082F006013C3EB13FBEA13FAEC14146007C3EB6A
:10083F0013FBEA13FA12075F883E893F22E54760F0
:10084F0034C3E53E9523F8E53F9400F9500CC3E817
:10085F009480E994FF4016020880C3E8947FE994DE
:0F086F00005003020880787F79000208807880AB
:10087E0079FF8843894422E5476058E5432540F8CF
:10088E00E5443541F9854420E4300701F43542FA58
:10089E0030E709C3EA94F040150208C2C3EA940F88
:1008AE0050030208C278FF79FF7A0F0208C278005F
:1008BE0079007AF0C3E524955E5006E524600901BF
:1008CE00DBE54420E70D01DBE54430E7068840898F
:1008DE00418A4222E547700302094678A1E6FAC32F
:1008EE00E54333F8E54433F9120797E930E70BC3D4
:1008FE00E89480E994FF4013211DC3E8947FE994A6
:10090E00005002211D787F7900211D788079FFE843
:10091E0020E715C3E52398F84009C3E89401400386
:10092E000209447801020944E8F424012523F84021
:10093E000302094478FF884522E54770030209A99E
:10094E0078A2E6FAA841A942120797E930E70CC34C
:10095E00E89401E994FF4016020980C3E894FFE988
:10096E009400500302098078FF7900020980780113
:10097E0079FFE920E715C3E54598F84009C3E894E7
:10098E000140030209A778000209A7E8F424012513
:10099E0045F840030209A778FF88242278FFC26435
:1009AE00E52D5406702FD264C3E53B940A4009C36B
:1009BE00E52594405002C264E53B601974FF853B07
:1009CE00F0848537F0A4F8C5F0600278FFC3E8958F
:1009DE00615002A8618860227883E6F520120F0428
:1009EE0075E8901206C675E890E5E820ECFBA8BD08
:1009FE00A9BE120F9A756BAB756C01C3740113FD12
:100A0E0074AB13FC74AB2CFC74013DFDECFAEDFBE6
:100A1E00C3E89AE99B4014E56B24ABF56BE56C34A7
:100A2E0001F56CEA2CFAEB3DFB80E5AE6BAF6CC3C7
:100A3E00E56C13F9E56B13F8C3E913F9E813F8E560
:100A4E006B28F569E56C39F56A7A03C3E913F9E8A1
:100A5E0013F8DAF7AA201A7009756B00756C00028C
:100A6E000A801AEA6008EE28FEEF39FFDAF88E6B7C
:100A7E008F6C2275E890227883E6FFE5E820ECF78C
:100A8E00A8BDA9BE056DC3E56D94084052756D00F5
:100A9E00E9FA79A0E76044EA7007E56E601B020A86
:100AAE00BBC3E8956E6010E56E5006600C14020A2A
:100ABE00C70460F9020AC7E56EF56EC394F6401BD3
:100ACE00755EC0C394064013755E80C39406400BDA
:100ADE00755E40C394064003755E0075BB0622EF3B
:100AEE00C39401601BC3E894FFE994035012C3E85A
:100AFE00956BE9956C5009E55E601A155E020B2345
:100B0E00E55EF46010055E7888E6B40308E55E24C1
:100B1E00044002F55EA85EC3E524985002A824C3E3
:100B2E00E8955F400AA85FE55FF46003855F5E7934
:100B3E0082B70402614EC3E895604002A860882522
:100B4E00E56DB4070375BB1022743279A387F0A448
:100B5E00C5F0A2F733F8C3E8955E4002A85E88227E
:100B6E0088248825886122753A00753B7F2275C8D6
:100B7E0020A8CCA9CD75C824AA38AB3988388939B4
:100B8E00C3E89AF8E99BF9AA3AAB3BAC3AAD3B7E87
:100B9E00047F02C3EB940440021E1FC3EB94084073
:100BAE00021E1FC3ED13FDEC13FCDEF7C3EA9CFA25
:100BBE00EB9DFBEF6009C3E913F9E813F8DFF7EAE1
:100BCE0028FAEB39FB8A3A8B3B400122753AFF75C6
:100BDE003BFF2230600261E1854C50854D51D26061
:100BEE0043E680227892E6FFC3E535948240010FFA
:100BFE00C3E53594A040010FC3EF940640027F0574
:100C0E007E021E3072010EC3E53B940350060E0E9B
:100C1E003072010EC3E53B940250060E0E30720187
:100C2E000EA93BA83A7A04C3E913F9E813F8DAF7E8
:100C3E00C3E89EF8E99400F94009C3E89402E994E8
:100C4E000050047802E4F9E9FBE8FAC3E913FDE881
:100C5E0013FC884C894DC3EF94036037EF20E00DF1
:0F0C6E00E82CF8E93DF9ECFAEDFB020C8EE828D2
:100C7D00F8E939F9C3E89402F8E99400F97A02E445
:100C8D00FBC3EF9403400D8A4E8B4F884889498CE6
:100C9D004A8D4B22884E894F8A488B498C4A8D4B01
:100CAD002230600281AED26043E680E52D540660AD
:100CBD0027A83AA93BE53494085006E820E002A99C
:100CCD004D759100C3E498F594E499F595759104EB
:100CDD00D26053917F43E68022D265753D00752029
:100CED0000020CF9D265753D00752040E52D5406C6
:100CFD006002C265D2AF206005E53D60012278013A
:100D0D007A02C3E53B940540027802C3E53B940AA1
:100D1D0040027803C3E53B940F40027A0330690427
:100D2D00781E7A01206007E53D6003D2AF22D2AF75
:100D3D000000C2AFC3E53BFB940F40027B0FEB04F9
:100D4D003073012320620123F93069027982E58B2A
:100D5D00C39940D0053DEAFBE59BF45440B5200412
:100D6D00DBF6A19520650281F9C265759100AE3A59
:100D7D00AF3BC3E49EF594E49FF595759104D26065
:100D8D0053917F43E68081F930650281F9D895D280
:100D9D00AF2230690B0534206016753400020DBD8D
:100DAD0020600D20650A206B071581158102159FA6
:100DBD0022A84EA94F75910053917FC3E498F594E5
:100DCD00E499F595759104854850854951D2604354
:100DDD00E6802278003064053065027801E53575CE
:100DED00F007A4F9E5F028F5F0E9A2F013A2F1134C
:100DFD00A2F213F535C394785003753578C3E535F4
:100E0D0095364008D266C290C291C292306002C13E
:100E1D0019854A50854B51D26043E68022C2AFD22C
:100E2D0093D294D29530720B9001FF7405D5E0FDED
:100E3D00020E40207D02C293307D02C295759F1136
:100E4D00753C02020F7FC2AF207D02C292307D023F
:100E5D00C2903072179001DCD294207D02D2953071
:100E6D007D02D2937405D5E0FD020E7C90013F30DA
:100E7D006206E5256002D291207D03759F01307DCC
:100E8D0003759F21753C03020F7FC2AFD293D2949D
:100E9D00D29530720B9001B97405D5E0FD020EADFF
:100EAD00207D02C295307D02C293207D03759F2166
:100EBD00307D03759F01753C04020F7FC2AFC29157
:100ECD00307217900196207D02D293307D02D2951B
:100EDD00D2947405D5E0FD020EEA90012D30620E1C
:100EED00E525600A207D02D290307D02D292759F59
:100EFD0011753C05020F7FC2AFD293D294D29530BB
:100F0D00720B90016B7405D5E0FD020F1AC294208F
:100F1D007D03759F01307D03759F21753C06020F82
:100F2D007FC2AF207D02C290307D02C29230721F0F
:100F3D0090022A207D02D293307D02D295207D022F
:100F4D00D295307D02D2937405D5E0FD020F5F90EE
:100F5D00015130620EE525600A207D02D292307D6E
:100F6D0002D290207D03759F21307D03759F017501
:100F7D003C01306B13120F9A7405D5E0FD7401D549
:100F8D00E0FDC293C294C295C266D2AF2290012BEE
:100F9D00C290C291C292D293D294D295C26222785B
:100FAD008076090876090876040876010876030824
:100FBD0076FF08760B087601087601087601788CA5
:100FCD0076010876FF0876FF0876FF0876FF08762B
:100FDD00FF0876030876FF0876FF0876FF0876256A
:100FED000876D00876280876500876040876FF082B
:100FFD00760208760008767A0876FF087601227860
:10100D0087E6FFC272BF0302D2727888E6C39403EB
:10101D006008C27DE630E102D27DC27E7889E6307D
:10102D00E102D27EC3EF94026008758E01D2730285
:10103D001044758E00C273227880E6149000809360
:10104D0078A1F67881E6149000809378A2F6120FBD
:10105D009A227886E61490008D9378A3F6120F9A53
:0E106D002222789CE67536FF75370CB4020619
:10107B007536A075370AB4030675368275370522A7
:10108B00227896E6FA7897E6FB307F047A007BFFAE
:10109B00C3EB9AFCC3948250027C82756F00056F80
:1010AB00EC856FF0A4C3E5F0948040F222D27F115F
:1010BB008C1206D57A007B007C101206CBE5592AE0
:1010CB00FA74003BFBDCF37C04C3EB13FBEA13FA6F
:1010DB00DCF7FEC27F118C22E5EF20E603752000C2
:1010EB000520903FFFE520146006901DFF14600063
:1010FB009304600375EF10C2D353D9BF7581C043FE
:10110B00FF801206C675EF0043B203E5B32404203B
:10111B00E702F5B3120F9A7580FF75A40075F19075
:10112B0075D47F75903875A53F75F23F75D50075F1
:10113B00A60175E241120FAC1215D078988670C2D9
:10114B00AF1206DF1206EF1206D51206F61206D5FF
:10115B001206FD1206D5C2AFE4F8F6D8FD78C879B1
:10116B00C8308707D9FBD8F7021C00120FAC121539
:10117B00D0110C1145115F116E116F118B118C7801
:10118B00988670120F9A75885075891275C82475D8
:10119B00910475D84075A82275B80275E690759BB9
:1011AB0080759D0075D10775BC5875BB0675BA1156
:1011BB0075E8801206C6D2AF1209E643DA01C2D82F
:1011CB00C2711206DF753001D2617B037A0CE558D0
:1011DB0070067A0CDB0221611206D52070022161A8
:1011EB00C270E559C3940240E3E52F541F855B5A47
:1011FB00F55BB55AD7DAD7C26153DACF207E0343FA
:10120B00DA20307E0343DA10C2D8C271C27575285A
:10121B00001206DA307409C3E528940A4002D2752D
:10122B001206CB78023074027800C3E5599840F06F
:10123B00C2AF1206EF1206EF1206EFD2AF1206DFA5
:10124B007546007888E6B40302612A1206CB788CC7
:10125B00E6C39401500302132AE530C394015003F3
:10126B0002132A207435C3E55994FF500302132A45
:10127B00C2AF120704D2AF1206DAC3E5599401507C
:10128B00EFC2AF1206EF1206D01206EFD2AF120664
:10129B00DAC3E55994FF40E90217787F02D27F1138
:1012AB008C1206DAC2AFC27F118CAE59C3E55994CA
:1012BB007FD2AF40741206C6C2AF120704D2AFDFA3
:1012CB00DC11B8C3EE94057897F61206DF121612EE
:1012DB001216FB7F0AD27F118C1206DAC2AFC27FC5
:1012EB00118CAE59C3E559947FD2AF50E61206C6A6
:1012FB00C2AF1206EF1206D01206EFD2AFDFD61135
:10130B00B8EE24057896F61206DF12161212172A7B
:10131B001206DA118CC3E55994FF40F4021778C317
:10132B00E559954640038559461206DA78017988C6
:10133B00E7B403027805C3E559984002414EC2AFAA
:10134B00120704120704120704D2AF1206DF75301E
:10135B0000E4F531F5320531E531F47039053278B9
:10136B009AE67819146012783214600D787D146047
:10137B000878FA146003753200C3E53298401715EC
:10138B00327531B478998670C2AF120704D2AF7838
:10139B009886701206DA1206D0E5297005307402B1
:1013AB00216178012074027806C3E5599840A7782B
:1013BB0088E6C3940360031206DAE5297002216103
:1013CB00C2AF120F9AE4F522F523F524F525D2AF1F
:1013DB0078858662F53EF53FF540F541F542F56DB2
:1013EB00F547F52CF52DF535120B75756D0875BB9D
:1013FB00101206C6120A81E5E820ECFBA8BDA9BEB7
:10140B00E97001F8886E120A85756D0875BB107846
:10141B0087E6FE7602110C7887EEF6C2AF755EFF9B
:10142B00120B5785225E85225F852260D2AF752213
:10143B0001752401752501855D64756501D268D23E
:10144B0069753400120F04120F2E120B75120B7CE0
:10145B00120BF202146C120F9A110C756D0075BB06
:0D146B0006120CF1120D9F120DBE1207EEBD
:10147800120DE0120E2A120B7C120BE1120BF21263
:101488000CAE120CE6120D9F120DBE12084C12097A
:10149800AA120DE0120E53120B7C120BE1120BF282
:1014A800120CAE120CF1120D9F120DBE120885120D
:1014B8000DE0120E97120B7C120BE1120BF2120CBC
:1014C800AE120CE6120D9F120DBE1208E2120DE0CC
:1014D800120EC9120B7C120BE1120BF2120CAE1297
:1014E8000CF1120D9F120DBE120947120DE0120FDA
:1014F80004120B7C120BE1120BF2120CAE120CE66A
:10150800120A81120D9F120DBE120A85120DE012E9
:101518000F2E120B7C120BE1120BF2120CAE30697B
:1015280038206B3585615E85615F855D6475650111
:1015380079327A0AC3E534994012C269D26A8A3389
:1015480085615E755FFF756020021561C3E559947A
:1015580001400302146C02159F306A1E206B1BE5C4
:1015680033147007C26A755EFF8161F533C3E559AC
:101578009401400302146C02159FC3E55C94FA5071
:1015880016307404E529600FC3E53B78F0306B0230
:101598007860985002816CC2AF120F9A7887E6FE85
:1015A8007602110C7887EEF6E4F522F523F524F59A
:1015B80025F562C268D2AF1206C6120F9A307406B9
:1015C800E52970022161615C901A0D782012165489
:1015D800E520B4550CA3121654E520B4AA0302154D
:1015E800F2120FAC121612021611901A0378807BB1
:1015F8000A121654A308DBF9901A0F788C7B15127F
:101608001654A308DBF9901A2422C2AF12169312BB
:10161800166D901A00740D121659A37402121659F9
:10162800A37413121659901A0378807B0A1216585D
:10163800A308DBF9901A0F788C7B15121658A308AB
:10164800DBF91216A6121684901A2422E493F622C5
:10165800E6438F01538FFD75EF0275B7A575B7F196
:10166800F0538FFE22438F02438F0175EF0275B747
:10167800A575B7F1901A0DF0538FFC22901A0D74CE
:1016880055D159901A0E74AAD159227A3079D07846
:1016980020901A40D154E520F709A3DAF7227A30CE
:1016A80079D0901A40E7D15909A3DAF922AB71A889
:1016B80072BB01027980BB02027981BB0302798285
:1016C800BB04027984BB05027983BB06027986BB19
:1016D80007027992BB08027987BB0902799CBB0A89
:1016E800027988BB0B027989E8F7227C051206DFAC
:1016F800DCFB22C2AF1206EF1206F61206FD120735
:10170800041206D01206EF1206F61206FD1207049E
:101718001206D01206EF1206F61206FD120704D2C0
:10172800AF22C2AF1207041206FD1206F61206EF28
:101738001206D01207041206FD1206F61206EF1260
:1017480006D01207041206FD1206F61206EFD2AFF3
:1017580022AE71AF72C2AF1206EF1206EF1206EF99
:101768001206D0DEF21207041206D0DFF8D2AF223A
:10177800D1FBD1F3D1F3757101757201757300F165
:10178800597C05AD591206DFC3ED955970F5C3E5CF
:10179800599401400AC3E55994FF40320217B4D165
:1017A800B5D112D1FBC2AF75EF10D1F3DCD50573FB
:1017B800C3E5739403500280C6D1F30572E5711432
:1017C80090009A93F808C3E57298500280AED1F35E
:1017D800D1F30571C3E571940C5002809C120FACD3
:0917E800D112C2AF75EF10D1F36C
:101A00000D02130909040103FF0B01010155AA018D
:101A1000FFFFFFFFFF03FFFFFF25D0285004FF0259
:051A2000007AFF01FF48
:101A400023585033412320202020202020202020F4
:101A500023424C48454C4923463333302320202031
:101A60002020202020202020202020202020202076
:101C0000C2AFC2D353D9BF7581C043B20343FF8073
:101C1000752438752503B1BF75EF0275E24043F1B5
:101C20008053A47FD287780379E67C1075220075F3
:101C30002300901DCC7B0675249875250130870202
:101C4000813D208708D8FBD9F9DCF781AD308708C2
:101C5000D8FBD9F9DCF781ADB17FE493A3C39A60D7
:101C6000028126DBDDB171600281267B08E493FAF4
:101C7000A3B152DBF87A30B152752200752300B15E
:101C800071EAFCEBFDC3ED94FE400EB1718A278B27
:101C900028ED30E0048A828B83B1717AC270D8C398
:101CA000ED94FE601050CEBD0022EC600675200061
:101CB0000200008100A827A9280809D804D90281B8
:101CC000C9B175EA89AAF281BB0D8199C3ED94036C
:101CD0005049EDA2E092007AC5C3E5829400E58305
:101CE000941C5093200010438F02438F0175B7A5B9
:101CF00075B7F1F030001FA827A9280809438F0104
:101D0000538FFDD804D902A11689AAE275B7A5752B
:101D1000B7F1F0A3A103538FFC81757AC1BD030C09
:101D2000E493A3FAB136DCF8B12E81758177AA224B
:101D3000AB23B152EBFAEA6222752608C3E52313FE
:101D4000F523E52213F52250066323A0632201D573
:101D500026EAB1BFB1BF75260AEAF4200102D28794
:101D6000300102C287B1BFC3134002C201D526EBC6
:101D700022B175EAFB208702A175308702A17A752E
:101D80002608AE24AF25C3EF13FFEE13FEB1C3B197
:101D9000BFC3EA133087024480FA30E703632201AD
:101DA000C3E52313F523E52213F52250066323A090
:101DB000632201D526D9E52265236523F52222AECB
:101DC00024AF250E0FDEFEDFFCD20122424C486517
:0A1DD0006C6934373132F33006013C
:00000001FF
